:0200000480007A
:10000000930E1000971000009380C0A3739050309F
:1000100097100000938080A673905010B71001F0E5
:100020001301000023A020001300000013000000B3
:100030001300000013000000130000001300000074
:100040001300000013000000130E1000170F000033
:10005000130FCF0073000000130E2000B720000024
:10006000938000801301000073B0003073200130D2
:10007000970000009380400173901034730020308B
:100080006F00901A170F0000130F4F02730000004B
:100090006F009019130E3000170F0000130F0F019F
:1000A000832010006F005018130E4000B72000008E
:1000B00093800080371100001301018073B000307D
:1000C000732001309700000093804001739010343A
:1000D000730020306F005015170F0000130F0F0131
:1000E000832010006F005014130E5000B720000042
:1000F000938000801301000073B000307320013042
:1001000097000000938040017390103473002030FA
:100110006F009011170F0000130F0F0183201000C4
:100120006F009010130E6000930000017390203058
:10013000130E7000170F0000130F0F018320100023
:100140006F00900E130E8000170F0000130FCF03E7
:10015000B720000093800080371100001301018058
:1001600073B000307320013097000000938040018D
:1001700073901034730020306F00100B8320100038
:100180006F00900A130E9000170F0000130F8F03DB
:10019000B7200000938000801301000073B000308E
:1001A0007320013097000000938040017390103459
:1001B000730020306F005007832010006F00D006BE
:1001C000130EA000170F0000130FCF07B71001F098
:1001D0001301000023A02000130000001300000002
:1001E00013000000130000001300000013000000C3
:1001F0001300000013000000930080007390003093
:10020000B71000009380008073904030B71001F069
:100210001301100023A020001300000013000000B1
:100220001300000013000000130000001300000082
:100230001300000013000000730050106F00C07E18
:10024000130EB000170F0000130F8F0AB71001F044
:100250001301000023A02000130000001300000081
:100260001300000013000000130000001300000042
:100270001300000013000000930080007390003012
:10028000B71000009380008073904030B7200000CA
:1002900093800080371100001301018073B000309B
:1002A0007320013097000000938040017390103458
:1002B000730020306F004077B71001F01301100079
:1002C00023A0200013000000130000001300000012
:1002D00013000000130000001300000013000000D2
:1002E00013000000730050106F000074130EC00064
:1002F000170F0000130F4F0AB71001F01301000091
:1003000023A02000130000001300000013000000D1
:100310001300000013000000130000001300000091
:10032000130000009300800073900030B7100000AD
:100330009380008073904030B7200000938000804D
:100340001301000073B000307320013097000000EB
:100350009380400173901034730020306F00C06CA4
:10036000B71001F01301100023A0200013000000BB
:100370001300000013000000130000001300000031
:100380001300000013000000130000007300501061
:100390006F0080699300200073900010130EE0003E
:1003A000170F0000130F0F08B72001F01301000012
:1003B00023A0200013000000130000001300000021
:1003C00013000000130000001300000013000000E1
:1003D0001300000093002000739000309300002071
:1003E00073904030930E0000B72001F0130110000D
:1003F00023A02000130000001300000013000000E1
:1004000013000000130000001300000013000000A0
:1004100013000000930040069380F0FFE34E10FEAF
:10042000130EF000170F0000130F8F0AB72001F012
:100430001301000023A0200013000000130000009F
:100440001300000013000000130000001300000060
:100450001300000013000000930020007390003090
:100460009300002073904030B720000093800080FC
:10047000371100001301018073B000307320013088
:100480009700000093804001739010347300203077
:100490006F008059930E1000B72001F01301100077
:1004A00023A0200013000000130000001300000030
:1004B00013000000130000001300000013000000F0
:1004C00013000000730050106F000056130E00015F
:1004D000170F0000130F0F0AB72001F013010000DF
:1004E00023A02000130000001300000013000000F0
:1004F00013000000130000001300000013000000B0
:10050000130000009300200073900030930000203F
:1005100073904030B72000009380008013010000EA
:1005200073B00030732001309700000093804001C9
:1005300073901034730020306F00004FB72001F02B
:100540001301100023A0200013000000130000007E
:10055000130000001300000013000000130000004F
:100560001300000013000000730050106F00C04B18
:10057000130E10019300002073903030170F00000D
:10058000130F0F08B72001F01301000023A0200073
:10059000130000001300000013000000130000000F
:1005A00013000000130000001300000013000000FF
:1005B000930020007390003093000020739040302F
:1005C000930E0000B72001F01301100023A02000BB
:1005D00013000000130000001300000013000000CF
:1005E00013000000130000001300000013000000BF
:1005F000930040069380F0FFE34E10FE130E20019F
:10060000170F0000130F8F0AB72001F0130100002D
:1006100023A02000130000001300000013000000BE
:10062000130000001300000013000000130000007E
:10063000130000009300200073900030930000200E
:1006400073904030B7200000938000803711000085
:100650001301018073B00030732001309700000057
:100660009380400173901034730020306F00C03BC2
:10067000930E1000B72001F01301100023A02000FA
:10068000130000001300000013000000130000001E
:10069000130000001300000013000000130000000E
:1006A000730050106F004038130E3001170F000018
:1006B000130F0F0AB72001F01301000023A0200040
:1006C00013000000130000001300000013000000DE
:1006D00013000000130000001300000013000000CE
:1006E00093002000739000309300002073904030FE
:1006F000B7200000938000801301000073B0003029
:1007000073200130970000009380400173901034F3
:10071000730020306F004031B72001F0130110004A
:1007200023A02000130000001300000013000000AD
:10073000130000001300000013000000130000006D
:1007400013000000730050106F00002EB72001F05E
:100750001301000023A0200013000000130000007C
:10076000130000001300000013000000130000003D
:100770001300000013000000130E4001170F0000CB
:10078000130F0F039300200073900030930000209C
:1007900073904030930E00009300002073A040142B
:1007A000930040069380F0FFE34E10FE130E5001BD
:1007B000170F0000130F0F069300002073B04014B2
:1007C000930020007390003093000020739040301D
:1007D000B7200000938000803711000013010180D2
:1007E00073B0003073200130970000009380400107
:1007F00073901034730020306F000023930E1000AC
:100800009300002073A04014730050106F00C021AB
:10081000130E6001170F0000130F8F0593000020C7
:1008200073B04014930020007390003093000020B8
:10083000739040309300002073A04014B720000054
:10084000938000801301000073B0003073200130EA
:1008500097000000938040017390103473002030A3
:100860006F00801C730050106F00001C130E70018D
:10087000930E0000B72001F01301000023A0200018
:10088000130000001300000013000000130000001C
:10089000130000001300000013000000130000000C
:1008A0009300002073B04014F3214034B72001F0CE
:1008B0001301100023A0200013000000130000000B
:1008C00013000000130000001300000013000000DC
:1008D00013000000130000009300002073B04014C8
:1008E000F3214034B72001F01301000023A02000C1
:1008F00013000000130000001300000013000000AC
:10090000130000001300000013000000130000009B
:100910009300002073B04014F3214034B72001F05D
:100920001301000023A020001300000013000000AA
:10093000130000001300000013000000130000006B
:1009400013000000130000009300002073A0401467
:10095000F3214034B72001F01301100023A0200040
:10096000130000001300000013000000130000003B
:10097000130000001300000013000000130000002B
:100980009300002073A04014F3214034B72001F0FD
:100990001301000023A0200013000000130000003A
:1009A00013000000130000001300000013000000FB
:1009B0001300000013000000130E800193002000BC
:1009C00073A0403073A0403473A00030930E100029
:1009D000170F0000130FCF03B72000009380008093
:1009E000371100001301018073B000307320013013
:1009F0009700000093804001739010347300203002
:100A00006F008002730050106F000002130E9001FF
:100A1000170F0000130F4F01736004307300501064
:100A20006F0080006F000001370110F0130141F2E8
:100A30002320C101370110F0130101F2232001002E
:100A4000E3840EFEF3202034F3201034F320003032
:100A5000F32030349300000873B00030930020007E
:100A6000E38A1EFCB72000009380008073A0003052
:100A700073101F3473002030E3880EFAF320201423
:100A8000F3201014F3200010F32030147300000042
:100A9000130000001300000013000000130000000A
:080AA000130000001300000028
:040000058000000077
:00000001FF
